 Debug

 Timestamp is 54e2a597 (Mon Feb 16 20:21:11 2015)

 Preferred load address is 10000000

 Start         Length     Name                   Class
 0001:00000000 00001a88H .text                   CODE
 0001:00001a88 00000043H .text$x                 CODE
 0002:00000000 000000ecH .idata$5                DATA
 0002:000000ec 00000004H .CRT$XCA                DATA
 0002:000000f0 00000004H .CRT$XCZ                DATA
 0002:000000f4 00000004H .CRT$XIA                DATA
 0002:000000f8 00000004H .CRT$XIAA               DATA
 0002:000000fc 00000004H .CRT$XIC                DATA
 0002:00000100 00000004H .CRT$XIZ                DATA
 0002:00000110 00000ef0H .rdata                  DATA
 0002:00001000 0000006cH .rdata$debug            DATA
 0002:00001070 00000010H .rdata$sxdata           DATA
 0002:00001080 00000004H .rtc$IAA                DATA
 0002:00001084 00000004H .rtc$IZZ                DATA
 0002:00001088 00000004H .rtc$TAA                DATA
 0002:0000108c 00000004H .rtc$TZZ                DATA
 0002:00001090 000000d4H .xdata$x                DATA
 0002:00001164 0000003cH .idata$2                DATA
 0002:000011a0 00000014H .idata$3                DATA
 0002:000011b4 000000ecH .idata$4                DATA
 0002:000012a0 000003ccH .idata$6                DATA
 0002:00001670 000005edH .edata                  DATA
 0003:00000000 0000001cH .data                   DATA
 0003:00000020 0000042cH .bss                    DATA
 0004:00000000 00000058H .rsrc$01                DATA
 0004:00000060 00000180H .rsrc$02                DATA

  Address         Publics by Value              Rva+Base       Lib:Object

 0000:00000000       __except_list              00000000     <absolute>
 0000:00000004       ___safe_se_handler_count   00000004     <absolute>
 0000:00009876       __ldused                   00009876     <absolute>
 0000:00009876       __fltused                  00009876     <absolute>
 0000:00000000       ___ImageBase               10000000     <linker-defined>
 0001:00000000       ?dbSetWarningID@@YGXXZ     10001000 f   dbExt.obj
 0001:00000081       ?dbSetWarningToTracefAux@@YGX_N@Z 10001081 f   dbExt.obj
 0001:00000090       _DllMain@12                10001090 f   Interface.obj
 0001:000000c9       ??0dbTraceObj@@QAE@ABV0@@Z 100010c9 f   db1.obj
 0001:00000109       ??0dbTraceObj@@QAE@XZ      10001109 f   db1.obj
 0001:0000013f       ??1dbTraceObj@@QAE@XZ      1000113f f   db1.obj
 0001:00000144       ??4dbTraceObj@@QAEAAV0@ABV0@@Z 10001144 f   db1.obj
 0001:00000171       ??8dbTraceObj@@QBE_NABV0@@Z 10001171 f   db1.obj
 0001:0000019e       ?Depth@dbTraceObj@@QBEIXZ  1000119e f   db1.obj
 0001:000001a1       ?FunctionAt@dbTraceObj@@QBEPBDI@Z 100011a1 f   db1.obj
 0001:0000022b       ?GenerateTrace@dbTraceObj@@SG?AV1@I@Z 1000122b f   db1.obj
 0001:0000028b       ?GetTraceAddress@dbTraceObj@@QBE?BJI@Z 1000128b f   db1.obj
 0001:000002a1       ?Release@dbTraceObj@@AAEXXZ 100012a1 f   db1.obj
 0001:000002f7       ?dbConvertAddress@@YG_NJPADI@Z 100012f7 f   db1.obj
 0001:00000391       ?dbConvertAddress@@YG_NJQAD00AAK@Z 10001391 f   db1.obj
 0001:00000417       ?dbDoStackTrace@@YG_NPAJJJ@Z 10001417 f   db1.obj
 0001:00000471       ?dbDoStackTrace@@YG_NPAJJJPBU_EXCEPTION_POINTERS@@@Z 10001471 f   db1.obj
 0001:000004ce       ?dbFatalfAux@@YAXPBDZZ     100014ce f   db1.obj
 0001:00000651       ?dbFatalfAuxExpr@@YAX_NPBDZZ 10001651 f   db1.obj
 0001:000006af       ?dbIsDebuggerPresent@@YG_NXZ 100016af f   db1.obj
 0001:0000070d       ?dbOutputHandlerAdd@@YGXP6GXQAPBDIK@Z@Z 1000170d f   db1.obj
 0001:0000074e       ?dbOutputHandlerRmv@@YGXP6GXQAPBDIK@Z@Z 1000174e f   db1.obj
 0001:000007f2       ?dbPrintStackTrace@@YGXABVdbTraceObj@@PBD@Z 100017f2 f   db1.obj
 0001:0000084e       ?dbSaveMiniDump@@YG_NPBDPBU_EXCEPTION_POINTERS@@@Z 1000184e f   db1.obj
 0001:0000085c       ?dbSilentErrors@@YGX_N@Z   1000185c f   db1.obj
 0001:0000086b       ?dbTraceHandlerAdd@@YGXP6GXQAPBDIK@Z@Z 1000186b f   db1.obj
 0001:000008ac       ?dbTraceHandlerRmv@@YGXP6GXQAPBDIK@Z@Z 100018ac f   db1.obj
 0001:00000903       ?dbTracefAux@@YAXPBDZZ     10001903 f   db1.obj
 0001:0000093a       ?dbTracefAuxExpr@@YAX_NPBDZZ 1000193a f   db1.obj
 0001:00000970       ?dbTracefAuxNS@@YAXPBDZZ   10001970 f   db1.obj
 0001:000009a0       ?dbWarningHandlerAdd@@YGXKP6GXQAPBDIK@Z@Z 100019a0 f   db1.obj
 0001:000009f3       ?dbWarningHandlerRmv@@YGXKP6GXQAPBDIK@Z@Z 100019f3 f   db1.obj
 0001:00000a35       ?dbWarningfAux@@YAXKPBDZZ  10001a35 f   db1.obj
 0001:00000ae0       ?dbWarningfAuxExpr@@YAX_NKPBDZZ 10001ae0 f   db1.obj
 0001:00000b1a       ?dbAddrLRUAddAddress@@YGXJPBD00K@Z 10001b1a f   dbAddrLRU1.obj
 0001:00000b1d       ?dbAddrLRUConvertAddress@@YG_NJQAD00AAK@Z 10001b1d f   dbAddrLRU1.obj
 0001:00000b22       ?dbAddrLRUSetup@@YGXXZ     10001b22 f   dbAddrLRU1.obj
 0001:00000b22       ?dbAddrLRUShutdown@@YGXXZ  10001b22 f   dbAddrLRU1.obj
 0001:00000b23       ?dbFree@@YGXPAX@Z          10001b23 f   dbCRT1.obj
 0001:00000b3c       ?dbMalloc@@YGPAXI@Z        10001b3c f   dbCRT1.obj
 0001:00000b55       ?dbModuleName@@YGXQADPBD@Z 10001b55 f   dbCRT1.obj
 0001:00000bb2       ?dbTrimTrailing@@YGXPAD@Z  10001bb2 f   dbCRT1.obj
 0001:00000be3       ?dbstrrchr@@YGPBDPBDD@Z    10001be3 f   dbCRT1.obj
 0001:00000cf4       ?dbSymGetSymFromAddr@@YG_NJQAD00AAK@Z 10001cf4 f   dbSymbols1.obj
 0001:00000e25       ?dbSymLoadDll@@YG_NXZ      10001e25 f   dbSymbols1.obj
 0001:00000f25       ?dbSymSaveMiniDump@@YG_NPBDPBU_EXCEPTION_POINTERS@@@Z 10001f25 f   dbSymbols1.obj
 0001:00000fdc       ?dbSymStackWalk@@YG_NQAJI@Z 10001fdc f   dbSymbols1.obj
 0001:0000101b       ?dbSymStackWalkException@@YG_NQAJIPBU_EXCEPTION_POINTERS@@@Z 1000201b f   dbSymbols1.obj
 0001:00001120       _memcmp                    10002120 f   MSVCRT:MSVCR110.dll
 0001:00001128       __EH_prolog                10002128 f   MSVCRT:ehprolog.obj
 0001:00001148       ___CxxFrameHandler3        10002148 f   MSVCRT:MSVCR110.dll
 0001:0000114e       _memset                    1000214e f   MSVCRT:MSVCR110.dll
 0001:00001160       __SEH_prolog               10002160 f   MSVCRT:sehprolg.obj
 0001:0000119b       __SEH_epilog               1000219b f   MSVCRT:sehprolg.obj
 0001:000011ac       __except_handler3          100021ac f   MSVCRT:MSVCR110.dll
 0001:000011fe       __CRT_INIT@12              100021fe f   MSVCRT:crtdll.obj
 0001:000013f3       __DllMainCRTStartup@12     100023f3 f   MSVCRT:crtdll.obj
 0001:0000154a       ___CppXcptFilter           1000254a f   MSVCRT:MSVCR110.dll
 0001:00001550       __amsg_exit                10002550 f   MSVCRT:MSVCR110.dll
 0001:00001560       __FindPESection            10002560 f   MSVCRT:pesect.obj
 0001:000015b0       __IsNonwritableInCurrentImage 100025b0 f   MSVCRT:pesect.obj
 0001:00001670       __ValidateImageBase        10002670 f   MSVCRT:pesect.obj
 0001:000016a1       ___atonexitinit            100026a1 f   MSVCRT:atonexit.obj
 0001:000016dd       __onexit                   100026dd f   MSVCRT:atonexit.obj
 0001:00001782       _atexit                    10002782 f   MSVCRT:atonexit.obj
 0001:00001797       ___security_init_cookie    10002797 f   MSVCRT:gs_support.obj
 0001:00001831       __RTC_Initialize           10002831 f   MSVCRT:initsect.obj
 0001:00001851       __RTC_Terminate            10002851 f   MSVCRT:initsect.obj
 0001:00001872       __initterm                 10002872 f   MSVCRT:MSVCR110.dll
 0001:00001878       __initterm_e               10002878 f   MSVCRT:MSVCR110.dll
 0001:0000187e       ___clean_type_info_names   1000287e f   MSVCRT:tncleanup.obj
 0001:00001890       __SEH_prolog4              10002890 f   MSVCRT:sehprolg4.obj
 0001:000018d5       __SEH_epilog4              100028d5 f   MSVCRT:sehprolg4.obj
 0001:000018e9       __except_handler4          100028e9 f   MSVCRT:chandler4gs.obj
 0001:0000190c       __lock                     1000290c f   MSVCRT:MSVCR110.dll
 0001:00001912       __unlock                   10002912 f   MSVCRT:MSVCR110.dll
 0001:00001918       ___dllonexit               10002918 f   MSVCRT:MSVCR110.dll
 0001:0000191e       ___clean_type_info_names_internal 1000291e f   MSVCRT:MSVCR110.dll
 0001:00001924       @__security_check_cookie@4 10002924 f   MSVCRT:secchk.obj
 0001:00001934       __except_handler4_common   10002934 f   MSVCRT:MSVCR110.dll
 0001:0000193a       ___raise_securityfailure   1000293a f   MSVCRT:gs_report.obj
 0001:00001977       ___report_gsfailure        10002977 f   MSVCRT:gs_report.obj
 0001:00001a70       __crt_debugger_hook        10002a70 f   MSVCRT:MSVCR110.dll
 0001:00001a76       ___crtUnhandledException   10002a76 f   MSVCRT:MSVCR110.dll
 0001:00001a7c       ___crtTerminateProcess     10002a7c f   MSVCRT:MSVCR110.dll
 0001:00001a82       _IsProcessorFeaturePresent@4 10002a82 f   kernel32:KERNEL32.dll
 0002:00000000       __imp__OutputDebugStringA@4 10003000     kernel32:KERNEL32.dll
 0002:00000004       __imp__GetProcAddress@8    10003004     kernel32:KERNEL32.dll
 0002:00000008       __imp__lstrcpyA@8          10003008     kernel32:KERNEL32.dll
 0002:0000000c       __imp__lstrcatA@8          1000300c     kernel32:KERNEL32.dll
 0002:00000010       __imp__lstrlenA@4          10003010     kernel32:KERNEL32.dll
 0002:00000014       __imp__LoadLibraryA@4      10003014     kernel32:KERNEL32.dll
 0002:00000018       __imp__HeapAlloc@12        10003018     kernel32:KERNEL32.dll
 0002:0000001c       __imp__HeapFree@12         1000301c     kernel32:KERNEL32.dll
 0002:00000020       __imp__GetProcessHeap@0    10003020     kernel32:KERNEL32.dll
 0002:00000024       __imp__lstrcpynA@12        10003024     kernel32:KERNEL32.dll
 0002:00000028       __imp__SetCurrentDirectoryA@4 10003028     kernel32:KERNEL32.dll
 0002:0000002c       __imp__GetCurrentDirectoryA@8 1000302c     kernel32:KERNEL32.dll
 0002:00000030       __imp__CreateFileA@28      10003030     kernel32:KERNEL32.dll
 0002:00000034       __imp__CloseHandle@4       10003034     kernel32:KERNEL32.dll
 0002:00000038       __imp__GetCurrentProcess@0 10003038     kernel32:KERNEL32.dll
 0002:0000003c       __imp__GetCurrentProcessId@0 1000303c     kernel32:KERNEL32.dll
 0002:00000040       __imp__GetCurrentThread@0  10003040     kernel32:KERNEL32.dll
 0002:00000044       __imp__GetCurrentThreadId@0 10003044     kernel32:KERNEL32.dll
 0002:00000048       __imp__OpenProcess@12      10003048     kernel32:KERNEL32.dll
 0002:0000004c       __imp__GetModuleFileNameA@12 1000304c     kernel32:KERNEL32.dll
 0002:00000050       __imp__IsDebuggerPresent@0 10003050     kernel32:KERNEL32.dll
 0002:00000054       __imp__GetSystemTimeAsFileTime@4 10003054     kernel32:KERNEL32.dll
 0002:00000058       __imp__QueryPerformanceCounter@4 10003058     kernel32:KERNEL32.dll
 0002:0000005c       __imp__DecodePointer@4     1000305c     kernel32:KERNEL32.dll
 0002:00000060       __imp__EncodePointer@4     10003060     kernel32:KERNEL32.dll
 0002:00000064       __imp__IsProcessorFeaturePresent@4 10003064     kernel32:KERNEL32.dll
 0002:00000068       \177KERNEL32_NULL_THUNK_DATA 10003068     kernel32:KERNEL32.dll
 0002:0000006c       __imp__memcmp              1000306c     MSVCRT:MSVCR110.dll
 0002:00000070       __imp__strchr              10003070     MSVCRT:MSVCR110.dll
 0002:00000074       __imp__getenv              10003074     MSVCRT:MSVCR110.dll
 0002:00000078       __imp___vsnprintf          10003078     MSVCRT:MSVCR110.dll
 0002:0000007c       __imp___controlfp          1000307c     MSVCRT:MSVCR110.dll
 0002:00000080       __imp____CxxFrameHandler3  10003080     MSVCRT:MSVCR110.dll
 0002:00000084       __imp__memset              10003084     MSVCRT:MSVCR110.dll
 0002:00000088       __imp___strlwr             10003088     MSVCRT:MSVCR110.dll
 0002:0000008c       __imp___except_handler3    1000308c     MSVCRT:MSVCR110.dll
 0002:00000090       __imp____CppXcptFilter     10003090     MSVCRT:MSVCR110.dll
 0002:00000094       __imp___amsg_exit          10003094     MSVCRT:MSVCR110.dll
 0002:00000098       __imp__free                10003098     MSVCRT:MSVCR110.dll
 0002:0000009c       __imp___malloc_crt         1000309c     MSVCRT:MSVCR110.dll
 0002:000000a0       __imp___initterm           100030a0     MSVCRT:MSVCR110.dll
 0002:000000a4       __imp___initterm_e         100030a4     MSVCRT:MSVCR110.dll
 0002:000000a8       __imp___lock               100030a8     MSVCRT:MSVCR110.dll
 0002:000000ac       __imp___unlock             100030ac     MSVCRT:MSVCR110.dll
 0002:000000b0       __imp___calloc_crt         100030b0     MSVCRT:MSVCR110.dll
 0002:000000b4       __imp____dllonexit         100030b4     MSVCRT:MSVCR110.dll
 0002:000000b8       __imp___onexit             100030b8     MSVCRT:MSVCR110.dll
 0002:000000bc       __imp____clean_type_info_names_internal 100030bc     MSVCRT:MSVCR110.dll
 0002:000000c0       __imp___except_handler4_common 100030c0     MSVCRT:MSVCR110.dll
 0002:000000c4       __imp___crt_debugger_hook  100030c4     MSVCRT:MSVCR110.dll
 0002:000000c8       __imp____crtUnhandledException 100030c8     MSVCRT:MSVCR110.dll
 0002:000000cc       __imp____crtTerminateProcess 100030cc     MSVCRT:MSVCR110.dll
 0002:000000d0       __imp___stricmp            100030d0     MSVCRT:MSVCR110.dll
 0002:000000d4       __imp___snprintf           100030d4     MSVCRT:MSVCR110.dll
 0002:000000d8       \177MSVCR110_NULL_THUNK_DATA 100030d8     MSVCRT:MSVCR110.dll
 0002:000000dc       __imp__GetActiveWindow@0   100030dc     user32:USER32.dll
 0002:000000e0       __imp__wsprintfA           100030e0     user32:USER32.dll
 0002:000000e4       __imp__MessageBoxA@16      100030e4     user32:USER32.dll
 0002:000000e8       \177USER32_NULL_THUNK_DATA 100030e8     user32:USER32.dll
 0002:000000ec       ___xc_a                    100030ec     MSVCRT:cinitexe.obj
 0002:000000f0       ___xc_z                    100030f0     MSVCRT:cinitexe.obj
 0002:000000f4       ___xi_a                    100030f4     MSVCRT:cinitexe.obj
 0002:00000100       ___xi_z                    10003100     MSVCRT:cinitexe.obj
 0002:00000e3c       ??_C@_08JMMIJEMM@USERNAME?$AA@ 10003e3c     dbExt.obj
 0002:00000e48       __real@3f800000            10003e48     Interface.obj
 0002:00000e4c       ??_C@_01EEMJAFIK@?6?$AA@   10003e4c     db1.obj
 0002:00000e50       ??_C@_02KFNNFDEI@?3?$CB?$AA@ 10003e50     db1.obj
 0002:00000e54       ??_C@_07IHMAFPOP@?$CFs?1?$CFd?$CFs?$AA@ 10003e54     db1.obj
 0002:00000e5c       ??_C@_0BB@EPBPNHDM@?9?9?5FATAL?5EXIT?5?9?9?$AA@ 10003e5c     db1.obj
 0002:00000e6d       ??_C@_00CNPNBAHC@?$AA@     10003e6d     db1.obj
 0002:00000e70       ??_C@_0BA@BGBOOLIN@?9?9stack?5trace?9?9?$AA@ 10003e70     db1.obj
 0002:00000e80       ??_C@_0BL@CKMAJDDL@0x?$CF08X?3?5?$CF?935s?5?5?5?5?5?5?5?5?5?$CI?$CFs?$CJ?$AA@ 10003e80     db1.obj
 0002:00000e9c       ??_C@_0BK@KMDBHLMD@0x?$CF08X?3?5?$CF?935s?5Ln?5?$CF4d?5?$CI?$CFs?$CJ?$AA@ 10003e9c     db1.obj
 0002:00000eb8       ??_C@_0N@HAOHNMDE@Kernel32?4dll?$AA@ 10003eb8     db1.obj
 0002:00000ec8       ??_C@_0BC@KNBMEBEO@IsDebuggerPresent?$AA@ 10003ec8     db1.obj
 0002:00000edc       ??_C@_0O@MCMFENKA@SymInitialize?$AA@ 10003edc     dbSymbols1.obj
 0002:00000eec       ??_C@_0L@GDMHENGB@SymCleanup?$AA@ 10003eec     dbSymbols1.obj
 0002:00000ef8       ??_C@_0BC@BDHGAJGO@SymGetSymFromAddr?$AA@ 10003ef8     dbSymbols1.obj
 0002:00000f0c       ??_C@_0BH@PMEMHADK@SymFunctionTableAccess?$AA@ 10003f0c     dbSymbols1.obj
 0002:00000f24       ??_C@_0BB@KAOAIDAF@SymGetModuleBase?$AA@ 10003f24     dbSymbols1.obj
 0002:00000f38       ??_C@_0O@LIDFOEPH@SymSetOptions?$AA@ 10003f38     dbSymbols1.obj
 0002:00000f48       ??_C@_0BB@GPFBCLFD@SymGetModuleInfo?$AA@ 10003f48     dbSymbols1.obj
 0002:00000f5c       ??_C@_09OJFIDCEK@StackWalk?$AA@ 10003f5c     dbSymbols1.obj
 0002:00000f68       ??_C@_0BD@HHOPHPBF@SymGetLineFromAddr?$AA@ 10003f68     dbSymbols1.obj
 0002:00000f7c       ??_C@_0BC@MNIKNFKD@MiniDumpWriteDump?$AA@ 10003f7c     dbSymbols1.obj
 0002:00000f90       ??_C@_0M@OOEJBPPK@dbghelp?4dll?$AA@ 10003f90     dbSymbols1.obj
 0002:00000f9c       ??_C@_0N@HNIPOBLH@imagehlp?4dll?$AA@ 10003f9c     dbSymbols1.obj
 0002:00000fac       __pRawDllMain              10003fac     MSVCRT:crtdll.obj
 0002:00000fac       __pDefaultRawDllMain       10003fac     MSVCRT:crtdll.obj
 0002:00000fb8       __load_config_used         10003fb8     MSVCRT:loadcfg.obj
 0002:00001070       ___safe_se_handler_table   10004070     <linker-defined>
 0002:00001080       ___rtc_iaa                 10004080     MSVCRT:initsect.obj
 0002:00001084       ___rtc_izz                 10004084     MSVCRT:initsect.obj
 0002:00001088       ___rtc_taa                 10004088     MSVCRT:initsect.obj
 0002:0000108c       ___rtc_tzz                 1000408c     MSVCRT:initsect.obj
 0002:00001164       __IMPORT_DESCRIPTOR_KERNEL32 10004164     kernel32:KERNEL32.dll
 0002:00001178       __IMPORT_DESCRIPTOR_USER32 10004178     user32:USER32.dll
 0002:0000118c       __IMPORT_DESCRIPTOR_MSVCR110 1000418c     MSVCRT:MSVCR110.dll
 0002:000011a0       __NULL_IMPORT_DESCRIPTOR   100041a0     kernel32:KERNEL32.dll
 0003:00000010       ___native_dllmain_reason   10005010     MSVCRT:natstart.obj
 0003:00000014       ___security_cookie         10005014     MSVCRT:gs_cookie.obj
 0003:00000018       ___security_cookie_complement 10005018     MSVCRT:gs_cookie.obj
 0003:00000020       ?g_silentErrors@@3_NA      10005020     db1.obj
 0003:00000021       ?g_useTracef@@3_NA         10005021     db1.obj
 0003:00000024       ?g_warningID@@3KA          10005024     db1.obj
 0003:00000028       ?s_dbStringOutputCB@?A0x64e34612@@3PAP6GXQAPBDIK@ZA 10005028     db1.obj
 0003:00000050       ?s_dbTraceStringOutputCB@?A0x64e34612@@3PAP6GXQAPBDIK@ZA 10005050     db1.obj
 0003:00000078       ?s_dbWarningStringOutputCB@?A0x64e34612@@3PAUdbWarnCB@1@A 10005078     db1.obj
 0003:000000c8       ?g_dbFilename@@3PBDB       100050c8     db1.obj
 0003:000000cc       ?g_dbLineNum@@3KA          100050cc     db1.obj
 0003:00000104       ___@@_PchSym_@00@UsrxplibRkxhsrkUslnvdliowCxozhhrxUhixUrmgvinvwrzgvUhszivwUwvyftUivovzhvUlyqUkxsBOlyq@AF5838954553F46D 10005104     pch1.obj
 0003:0000010c       ?__type_info_root_node@@3U__type_info_node@@A 1000510c     MSVCRT:tncleanup.obj
 0003:00000438       ___native_startup_lock     10005438     <common>
 0003:0000043c       ___native_startup_state    1000543c     <common>
 0003:00000440       ___onexitend               10005440     <common>
 0003:00000444       ___onexitbegin             10005444     <common>
 0003:00000448       ___dyn_tls_init_callback   10005448     <common>

 entry point at        0001:000013f3

 Static symbols

 0000:ffff8000       .debug$S                   10000000     kernel32:KERNEL32.dll
 0000:ffff8000       .debug$S                   10000000     MSVCRT:MSVCR110.dll
 0000:ffff8000       .debug$S                   10000000     MSVCRT:MSVCR110.dll
 0000:ffff8000       .debug$S                   10000000     MSVCRT:MSVCR110.dll
 0000:ffff8000       .debug$S                   10000000     MSVCRT:MSVCR110.dll
 0000:ffff8000       .debug$S                   10000000     MSVCRT:MSVCR110.dll
 0000:ffff8000       .debug$S                   10000000     MSVCRT:MSVCR110.dll
 0000:ffff8000       .debug$S                   10000000     MSVCRT:MSVCR110.dll
 0000:ffff8000       .debug$S                   10000000     MSVCRT:MSVCR110.dll
 0000:ffff8000       .debug$S                   10000000     MSVCRT:MSVCR110.dll
 0000:ffff8000       .debug$S                   10000000     MSVCRT:MSVCR110.dll
 0000:ffff8000       .debug$S                   10000000     MSVCRT:MSVCR110.dll
 0000:ffff8000       .debug$S                   10000000     MSVCRT:MSVCR110.dll
 0000:ffff8000       .debug$S                   10000000     MSVCRT:MSVCR110.dll
 0000:ffff8000       .debug$S                   10000000     MSVCRT:MSVCR110.dll
 0000:ffff8000       .debug$S                   10000000     MSVCRT:MSVCR110.dll
 0000:ffff8000       .debug$S                   10000000     MSVCRT:MSVCR110.dll
 0000:ffff8000       .debug$S                   10000000     MSVCRT:MSVCR110.dll
 0000:ffff8000       .debug$S                   10000000     MSVCRT:MSVCR110.dll
 0000:ffff8000       .debug$S                   10000000     MSVCRT:MSVCR110.dll
 0000:ffff8000       .debug$S                   10000000     MSVCRT:MSVCR110.dll
 0000:ffff8000       .debug$S                   10000000     MSVCRT:MSVCR110.dll
 0000:ffff8000       .debug$S                   10000000     MSVCRT:MSVCR110.dll
 0000:ffff8000       .debug$S                   10000000     MSVCRT:MSVCR110.dll
 0000:ffff8000       .debug$S                   10000000     MSVCRT:MSVCR110.dll
 0000:ffff8000       .debug$S                   10000000     MSVCRT:MSVCR110.dll
 0000:ffff8000       .debug$S                   10000000     MSVCRT:MSVCR110.dll
 0000:ffff8000       .debug$S                   10000000     user32:USER32.dll
 0000:ffff8000       .debug$S                   10000000     user32:USER32.dll
 0000:ffff8000       .debug$S                   10000000     user32:USER32.dll
 0000:ffff8000       .debug$S                   10000000     kernel32:KERNEL32.dll
 0000:ffff8000       .debug$S                   10000000     kernel32:KERNEL32.dll
 0000:ffff8000       .debug$S                   10000000     kernel32:KERNEL32.dll
 0000:ffff8000       .debug$S                   10000000     kernel32:KERNEL32.dll
 0000:ffff8000       .debug$S                   10000000     kernel32:KERNEL32.dll
 0000:ffff8000       .debug$S                   10000000     kernel32:KERNEL32.dll
 0000:ffff8000       .debug$S                   10000000     kernel32:KERNEL32.dll
 0000:ffff8000       .debug$S                   10000000     kernel32:KERNEL32.dll
 0000:ffff8000       .debug$S                   10000000     kernel32:KERNEL32.dll
 0000:ffff8000       .debug$S                   10000000     kernel32:KERNEL32.dll
 0000:ffff8000       .debug$S                   10000000     kernel32:KERNEL32.dll
 0000:ffff8000       .debug$S                   10000000     kernel32:KERNEL32.dll
 0000:ffff8000       .debug$S                   10000000     kernel32:KERNEL32.dll
 0000:ffff8000       .debug$S                   10000000     kernel32:KERNEL32.dll
 0000:ffff8000       .debug$S                   10000000     kernel32:KERNEL32.dll
 0000:ffff8000       .debug$S                   10000000     kernel32:KERNEL32.dll
 0000:ffff8000       .debug$S                   10000000     kernel32:KERNEL32.dll
 0000:ffff8000       .debug$S                   10000000     kernel32:KERNEL32.dll
 0000:ffff8000       .debug$S                   10000000     kernel32:KERNEL32.dll
 0000:ffff8000       .debug$S                   10000000     kernel32:KERNEL32.dll
 0000:ffff8000       .debug$S                   10000000     kernel32:KERNEL32.dll
 0000:ffff8000       .debug$S                   10000000     kernel32:KERNEL32.dll
 0000:ffff8000       .debug$S                   10000000     kernel32:KERNEL32.dll
 0000:ffff8000       .debug$S                   10000000     kernel32:KERNEL32.dll
 0000:ffff8000       .debug$S                   10000000     kernel32:KERNEL32.dll
 0000:ffff8000       .debug$S                   10000000     MSVCRT:MSVCR110.dll
 0001:00000687       ?dbFormatf@@YGXQADIPBDPAD@Z 10001687 f   db1.obj
 0001:0000077c       ?dbPrintInternal@@YGXQAPBDI@Z 1000177c f   db1.obj
 0001:000008da       ?dbTraceInternal@@YGXQAPBDI@Z 100018da f   db1.obj
 0001:00000c10       ?MapFunctions@@YG_NPAUHINSTANCE__@@@Z 10001c10 f   dbSymbols1.obj
 0001:00001128       $$000000                   10002128     MSVCRT:ehprolog.obj
 0001:00001160       $$000000                   10002160     MSVCRT:sehprolg.obj
 0001:000011b2       _pre_c_init                100021b2 f   MSVCRT:crtdll.obj
 0001:00001416       ___DllMainCRTStartup       10002416 f   MSVCRT:crtdll.obj
 0001:00001890       $$000000                   10002890     MSVCRT:sehprolg4.obj
 0001:00001a88       __unwindfunclet$?GenerateTrace@dbTraceObj@@SG?AV1@I@Z$0 10002a88 f   db1.obj
 0001:00001aa1       __ehhandler$?GenerateTrace@dbTraceObj@@SG?AV1@I@Z 10002aa1 f   db1.obj
 0001:00001aab       __unwindfunclet$?dbFatalfAux@@YAXPBDZZ$0 10002aab f   db1.obj
 0001:00001ab6       __unwindfunclet$?dbFatalfAux@@YAXPBDZZ$1 10002ab6 f   db1.obj
 0001:00001ac1       __ehhandler$?dbFatalfAux@@YAXPBDZZ 10002ac1 f   db1.obj
 0002:000000f8       _pcinit                    100030f8     MSVCRT:crtdll.obj
 0002:000000fc       _pinit                     100030fc     MSVCRT:atonexit.obj
 0002:00000148       _artist                    10003148     dbExt.obj
 0002:00000940       _design                    10003940     dbExt.obj
 0002:00000fb0       _GS_ExceptionPointers      10003fb0     MSVCRT:gs_report.obj
 0002:00001090       __unwindtable$?dbFatalfAux@@YAXPBDZZ 10004090     db1.obj
 0002:000010a0       __ehfuncinfo$?dbFatalfAux@@YAXPBDZZ 100040a0     db1.obj
 0002:000010c4       __unwindtable$?GenerateTrace@dbTraceObj@@SG?AV1@I@Z 100040c4     db1.obj
 0002:000010cc       __ehfuncinfo$?GenerateTrace@dbTraceObj@@SG?AV1@I@Z 100040cc     db1.obj
 0002:000010f0       __sehtable$?dbSymStackWalk@@YG_NQAJI@Z 100040f0     dbSymbols1.obj
 0002:00001100       __sehtable$___DllMainCRTStartup 10004100     MSVCRT:crtdll.obj
 0002:00001128       __sehtable$__IsNonwritableInCurrentImage 10004128     MSVCRT:pesect.obj
 0002:00001148       __sehtable$__onexit        10004148     MSVCRT:atonexit.obj
 0002:000013f6       .idata$6                   100043f6     kernel32:KERNEL32.dll
 0002:00001430       .idata$6                   10004430     user32:USER32.dll
 0002:000014cc       .idata$6                   100044cc     MSVCRT:MSVCR110.dll
 0002:00001670       .edata                     10004670     Debug.exp
 0002:00001698       rgpv                       10004698     Debug.exp
 0002:00001724       rgszName                   10004724     Debug.exp
 0002:000017b0       rgwOrd                     100047b0     Debug.exp
 0002:000017f6       szName                     100047f6     Debug.exp
 0002:00001800       $N00001                    10004800     Debug.exp
 0002:0000181b       $N00002                    1000481b     Debug.exp
 0002:00001831       $N00003                    10004831     Debug.exp
 0002:00001847       $N00004                    10004847     Debug.exp
 0002:00001866       $N00005                    10004866     Debug.exp
 0002:00001882       $N00006                    10004882     Debug.exp
 0002:0000189c       $N00007                    1000489c     Debug.exp
 0002:000018be       $N00008                    100048be     Debug.exp
 0002:000018e4       $N00009                    100048e4     Debug.exp
 0002:0000190b       $N00010                    1000490b     Debug.exp
 0002:00001927       $N00011                    10004927     Debug.exp
 0002:00001946       $N00012                    10004946     Debug.exp
 0002:00001969       $N00013                    10004969     Debug.exp
 0002:00001986       $N00014                    10004986     Debug.exp
 0002:000019bb       $N00015                    100049bb     Debug.exp
 0002:000019d2       $N00016                    100049d2     Debug.exp
 0002:000019ef       $N00017                    100049ef     Debug.exp
 0002:00001a0c       $N00018                    10004a0c     Debug.exp
 0002:00001a34       $N00019                    10004a34     Debug.exp
 0002:00001a5c       $N00020                    10004a5c     Debug.exp
 0002:00001a88       $N00021                    10004a88     Debug.exp
 0002:00001abb       $N00022                    10004abb     Debug.exp
 0002:00001ad2       $N00023                    10004ad2     Debug.exp
 0002:00001af4       $N00024                    10004af4     Debug.exp
 0002:00001b0d       $N00025                    10004b0d     Debug.exp
 0002:00001b34       $N00026                    10004b34     Debug.exp
 0002:00001b5b       $N00027                    10004b5b     Debug.exp
 0002:00001b72       $N00028                    10004b72     Debug.exp
 0002:00001b8f       $N00029                    10004b8f     Debug.exp
 0002:00001ba8       $N00030                    10004ba8     Debug.exp
 0002:00001bd2       $N00031                    10004bd2     Debug.exp
 0002:00001bfc       $N00032                    10004bfc     Debug.exp
 0002:00001c16       $N00033                    10004c16     Debug.exp
 0002:00001c36       $N00034                    10004c36     Debug.exp
 0002:00001c4b       $N00035                    10004c4b     Debug.exp
 0003:00000000       ?crap@?1??DllMain@@9@12@4MA 10005000     Interface.obj
 0003:000000d0       ?pfnTest@?1??dbIsDebuggerPresent@@YG_NXZ@4_NA 100050d0     db1.obj
 0003:000000d4       ?pfn@?1??dbIsDebuggerPresent@@YG_NXZ@4P6GHXZA 100050d4     db1.obj
 0003:000000d8       _s_dbSymInitialized        100050d8     dbSymbols1.obj
 0003:000000dc       __SymInitialize            100050dc     dbSymbols1.obj
 0003:000000e0       __SymCleanup               100050e0     dbSymbols1.obj
 0003:000000e4       __SymGetSymFromAddr        100050e4     dbSymbols1.obj
 0003:000000e8       __SymGetLineFromAddr       100050e8     dbSymbols1.obj
 0003:000000ec       __SymFunctionTableAccess   100050ec     dbSymbols1.obj
 0003:000000f0       __SymGetModuleBase         100050f0     dbSymbols1.obj
 0003:000000f4       __SymSetOptions            100050f4     dbSymbols1.obj
 0003:000000f8       __SymGetModuleInfo         100050f8     dbSymbols1.obj
 0003:000000fc       __StackWalk                100050fc     dbSymbols1.obj
 0003:00000100       __MiniDumpWriteDump        10005100     dbSymbols1.obj
 0003:00000108       ___proc_attached           10005108     MSVCRT:crtdll.obj
 0003:00000118       _GS_ExceptionRecord        10005118     MSVCRT:gs_report.obj
 0003:00000168       _GS_ContextRecord          10005168     MSVCRT:gs_report.obj
 0003:00000434       _DebuggerWasPresent        10005434     MSVCRT:gs_report.obj
 0004:00000060       $R000000                   10006060     * linker generated manifest res *
